:100000000C9449050C9466050C9466050C946605E1
:100010000C9466050C9466050C9466050C946605B4
:100020000C9466050C9466050C9466050C946605A4
:100030000C9466050C9466050C9466050C94660594
:100040000C9466050C9466050C9466050C94660584
:100050000C9466050C9466050C9466050C94660574
:100060000C94680D0C946605A877A6E0F7435A3502
:1000700085E272978FB71A6287380D67C7BE4F3E09
:100080002076378F68B7A9263F2B10E3307E900E7D
:10009000850A70510386400D4FEB3ECCD18735BDAC
:1000A000F50B5ED0F8F2D5E26C310CADFC21C378D3
:1000B000C106C24C55E64A3448111EDAE71A84A03C
:1000C00096A7E37FAF639CFA235B79C89EBAB2C957
:1000D00022124BB3A1B63249A2E189391066C50795
:1000E0008F54EA91CA3FF919F0D746BC281B61E842
:1000F0002F6AAE9DF64E0914774DDB1F2E7B7CF1E7
:1001000043A300B8138C85B9297588FDD2561C50BD
:100110009741E53B60B5C064EE98D62D25A4AACDE5
:100120007DA883C6ABBE4499263CCE9FBFD3CB7679
:100130007A7E82018A9A801D0EB05CD43862F430D7
:10014000E08E53B70257ACA6520A6D92651724335E
:10015000457274B1B4F75DED2CFF47375A90BBDFA1
:100160002A165995D9C4276773C768FEA5DD6B5F4A
:1001700093D8EC053A8D6EFB3DA96936F394DEEF1A
:10018000156F8B9B080FDC81182004E471CFE92BDD
:10019000425801A0A962D63F85A7B6D4FA156617C2
:1001A00009BD5D14342659729154064FF8B05B7442
:1001B00093998CF245CDEA4EAD104AE5CAEEDFC602
:1001C0006F9F888E02CC08A877946D21B128E439FE
:1001D0007996607181162EE678B9C4469A42AEB718
:1001E0007C43B3221A86C2323D2D9CD229E9639BFF
:1001F000D131385E1E3641BB03182B3EBF6861FC0F
:1002000052C0DEE00A58135A00BE1C900E5312FD75
:10021000E26EBACE2427447F87A3A1D55040E3F9EC
:1002200083F7C7A235C8DB19AB2F1125ED339E55D7
:10023000E148AF7384DA2AAA51EB9D95B2CBE770FF
:1002400080FE4C6504EFC5F1C33AB4F55F2389DD48
:1002500030A58BD3F6DC4D64D7F08FEC56375CA419
:100260000D07768A2C0BB5D8C11FE83BF44B1B4712
:100270006C49677B92CF757E20D97D3C977AD005FB
:100280006B0F1DFB8298578DF36ABCACC9A6FFB8F3
:10029000690C4C4D72075A49338DA2AB463D630D34
:1002A000A097FFF0F5FAC0E9DB62E4E17443DC8675
:1002B000182937F406E2ED6F90481E2D1DEA73945D
:1002C00054DF25F64727D91177C9841C5B5C51811F
:1002D000A6223E2496C88AEC827C09B8454A57BBC0
:1002E0002F50758E61708C6CAFD0FDB41BAEDEFEEE
:1002F0003BB536BD55010E9C41565FB3260383BA0C
:10030000134BCAC50AF860A5B9C7C39832FB12F9E6
:10031000A792AA68F3787E05202102E8BFF2B059BF
:100320008FD2CB876515F11AB230ADEE58A38B662C
:100330001F2CD75D1985A8E6D36BA10C91936A5E3B
:100340000B79E3DD004F3C896E7169A9AC40E599FA
:1003500028C6314E7ACD089E7DEF17FC88D8A46D53
:100360004495D1B7D49BBE2A34642BCF2EEB38CE24
:1003700023E03A3FF77B9F1053BC526716E7807625
:1003800004C4B6C1C27F9ADAD53942149DB10F3583
:10039000D6CCB9DA380CA29C091F06B1B6FD1A6991
:1003A0002330C4DE01D1F45829371C7DD5BFFFBDF1
:1003B000C8C9CF65BE7B7897986708B32657F7FA08
:1003C00040AD8E75A67CDB918B5199D4177A908DB8
:1003D000CE63CB4EA0AB183A5B507F2174C1BBB843
:1003E000B7BA0B359531599A4D04071E5A7613F357
:1003F0007183D08603A83942AA28E6E4D85DD3D019
:100400006E6F96FB5EBC56C25F859BE7AFD23B84A6
:100410006AA753C54449A5F936723D2CD91BA1F5ED
:100420004F939D68474116CA2A4CA387D6E5192EDB
:1004300077156D70C0DFB20046EDC66C4360922D3B
:10044000A922458F3455AEA40A6632E0DC02ACE83E
:10045000208C89624AFEEEC3E33CF17905E9F62778
:1004600033CCF29E11817E80108A829F480DD7B4D2
:10047000FC2FB5C7DD88146B2B54EA1D945CB0EFDC
:100480001224CDEBE1E264733F0E5261253EF80F7A
:100490004BECC00030F602493D106E20C9A62FFE7D
:1004A0002C2B752E4526AB48A980FC04CCD3B5BABD
:1004B000A338317D01D9A77B96B663694EF7DEE09C
:1004C00078CA50AA41916588E42185DA3A27BE1C92
:1004D0003E425E17527F1F89246F8F5C67740E1235
:1004E000878DE934ED73C4F8615B05DF594C97796A
:1004F0008318A45595EBBD53F5F15766469FB2811D
:100500000951862216DD23937629C2D71DD4BF3622
:100510003FEA4B1132B9625460D66D439A0D929CFA
:10052000B0EF586C9D772D70FAF3B30BE2407EF478
:100530008AE58C3C5671D164E1820ACB131590ECAC
:100540000399AF145D0F334A94A5A8351BE36AC61F
:1005500028FF4DE72584AC08AEC5A22AB8370C7A2F
:10056000A0C3CEAD061A9E8BFBD5D0C11ED0B49BC6
:10057000B144F247C768CF72BB4F5AF9DC6BDBD28C
:10058000E87CC8EE98A1E6D839075FFD8E19B73B25
:10059000BCCD7CE38173B211BF6F2098FE7596EFDE
:1005A0006CDA50E109725445BA34805BED3E532C4D
:1005B00087A457F3333F3CB767B4A325604F076B5D
:1005C0001B47150FE40AEAD1327836498D4BD2BC6D
:1005D000A5DC1D0D4DCD9A825FFC9465BEE2F4C989
:1005E0001E44CB9E0C64712663B314E840708A0EDF
:1005F00019426DAC88105CDF41A9ADE5FB74CCD528
:10060000068E5986CE1F3D76E08FB977277BA6D818
:1006100029D3ECB813F7FAC3516ADE4A5AEBC28BFE
:10062000234892CF62A899F8D02E856143C8BDF0C7
:100630000593CA4EF17D30FDC469662F08B152F9A9
:1006400021E67A2BDD3984FFC091D637D47F2D9BEC
:100650005DA13B6EB5C54604F590EE7E831C035646
:10066000B6AA0017013555790B12BB1A31E70228DB
:1006700016C1F6A2DB189C89683897ABC72AD73A0F
:10068000F2C6244CB058A0225E9DD9A7E9AEAF8C2B
:10069000959F28B720D7B030C30919C067D6003C52
:1006A0007EE7E9F4085AF8B82E05A6259E5CD81511
:1006B0000DE1F611546BCD2146665E84AD063829F6
:1006C00044C5A2CEF1AAC1407186B5EFFC36A8CBD5
:1006D0000A48274564A3AF8CB2C69F0789DC17D3AD
:1006E0004979FBFE1DD0B9884352BC01782B7D941B
:1006F000C70EDEA5D59BCCF7617AC274813903ABF6
:1007000096A037BD2D72753FC9D48E6FF98DED62FD
:10071000DB1CDF04AC1B6C144B63D0BFB482EC7BDE
:100720001A5992D21060B63D5FE6806E70C4F23501
:10073000D97CEEE541A45B50DDBB4CF31F9D5D57BA
:10074000555197E358424D9C73BAC877316926AE2C
:10075000EA8ADA22B38756FA930B341633E8E45365
:10076000BEA9B13A3EF5906ACF3B12FD8F9AA747DA
:100770009199EB0F24FF2318854E7F0CE0A1D2D175
:100780002C2A4A024F1E95688B98836D76CA653273
:10079000132FC3829AA4BA8160373435FC80A851E4
:1007A0006567ED305F10D34A272F13B92AD2CCE109
:1007B000EFAEEBBEF4BDCF43B3C58884B7DD39409F
:1007C000CE486D9B72617EE7A14E532E773BE2C906
:1007D00036221B6E73B103B24C87A9D44D0FD815C6
:1007E0006CAA18F649575DFB7A149463A011B09E69
:1007F000DE0546C8EE47DBDC24899C919729E97B1E
:10080000C1071EB8FDFEACC662984FF179E0E86BF7
:100810007856B68D045086CA6F20E6EAE576171C36
:10082000747FBC0D2C85F76696E48B753F4BD938E9
:10083000AF7CDA0B832D3132A2F51D594145BF3C07
:100840001FF8F98AD016256912999D2195AB01A64A
:10085000D7B5C07DFF580E3A92D155E3089FD63EDA
:10086000528EFAA3C702CDDF8F64198CF3A70C5EFA
:100870000A6A09F0935B42C20623EC71ADB4CBBBAC
:100880007028D51A5C33685A004490A5C4263D2BC5
:10089000F25496ADDA1FED33E18169080D0ADB35BC
:1008A000779A64D1FC78AA1BD067A0DDFA6C6371DB
:1008B0000584176A894F667FC65055926FBDE7D28F
:1008C00040728DBBEC06428AE4889D7E7A822713B3
:1008D000411AAFC8A476B4C2FE6D1CD96130B37C96
:1008E000EAF7290FF23B51C1DE5FE52A2F990B5D34
:1008F000A32B4AAB95A5D35856EE283100CC15460C
:10090000CAE686383C65F5E39FD65B094983702DBE
:1009100053A97DE2C4AC8E5EB825F4B957F3F168F3
:1009200047B2A25920CE34795C900E1EBED5222348
:10093000B1C91862162E913E078FD83F933DD49BC4
:10094000DF8521FB117497C7D7DC4C194598E94323
:10095000024BBCC3049C6BF07552A726F6C5BACFF8
:10096000B0B7AE5AA1BF038B80126E0CEBF9C04436
:1009700024EF10F8A88CE87BFF9E2CCD603687B55D
:1009800094A654733A144E011DB6FD37484D39CB29
:10099000E032000000000000000000000000000045
:1009A0000000000000000000000000000000000047
:1009B0000000000000000000000000000000000037
:1009C0000000000000000000000000000000000027
:1009D0000000000000000000000000000000000017
:1009E0000000000000000000000000000000000007
:1009F00000000000000000000000000000000000F7
:100A000000000000000000000000000000000000E6
:100A100000000000000000000000000000000000D6
:100A200000000000000000000000000000000000C6
:100A300000000000000000000000000000000000B6
:100A400000000000000000000000000000000000A6
:100A50000000000000000000000000000000000096
:100A60000000000000000000000000000000000086
:100A70000000000000000000000000000000000076
:100A80000000000000000000000000000000000066
:100A9000000011241FBECFEFD4E0DEBFCDBF11E0B8
:100AA000A0E0B1E0EEE0F5E202C005900D92AC34BA
:100AB000B107D9F713E0ACE4B1E001C01D92A73C47
:100AC000B107E1F70E947A090C9485120C9400009A
:100AD000DC01FB01108617821482138212821182BC
:100AE0004C91433009F4DEC0443020F4423009F028
:100AF00051C307C0443009F4AAC1453009F04AC3C4
:100B000020C180914C0111969C911197882379F016
:100B100091FF04C080E490E09087878311968C91C8
:100B2000119780FF2AC087819085806124C090FF43
:100B300004C080E490E09087878311968C91119790
:100B400081FF05C087819085806290878783119699
:100B50008D919C91129790FF05C08781908580614F
:100B60009087878311968D919C91129791FF05C074
:100B70008781908588609087878380914D01119649
:100B80009C9111978823D1F094FF02C084E6828360
:100B900011968C91119785FF02C08CE98283119682
:100BA0008C91119786FF02C08CE9818311968C91FC
:100BB000119787FF28C084E6818325C094FF05C074
:100BC0008781908581609087878311968C9111979A
:100BD00085FF05C0878190859064908787831196F3
:100BE0008C91119786FF05C08781908582609087E0
:100BF000878311968C91119787FF05C08781908517
:100C000090689087878311968C91119782FF05C019
:100C10008781908590619087878311968C91119739
:100C200083FF05C0878190859460908787831196A4
:100C30008D919C91129792FF05C08781908590625B
:100C40009087878311968D919C91129793FF05C091
:100C50008781908592609087878311962D913C9132
:100C60001297C9018C719C708C519C4021F4109298
:100C70004C0110924D01C9018C729C708C529C40A9
:100C800029F481E080934C0110924D012C743C704A
:100C90002C543C4009F07EC281E080934D011092BB
:100CA0004C01089511968C91119780FF04C080E14A
:100CB00090E09087878311968C91119781FF05C0F2
:100CC0008781908580649087878311968C91119796
:100CD00082FF05C0878190859061908787831196F8
:100CE0008C91119783FF05C08781908594609087D0
:100CF000878311968C91119784FF05C08781908519
:100D000081609087878311968C91119785FF05C02C
:100D10008781908590649087878311968C91119735
:100D200086FF05C0878190858260908787831196B2
:100D30008C9187FF2FC287819085906890878783E9
:100D4000089517968C91179787FF04C080E190E073
:100D50009087878317968C91179786FF05C08781A8
:100D6000908580649087878317968C91179785FF6D
:100D700005C08781908588609087878317968C91BE
:100D8000179784FF05C0878190858062908787834D
:100D900017968D919C91189791FF05C0878190853A
:100DA00090629087878317968D919C91189792FFF8
:100DB00005C08781908592609087878317968C9174
:100DC000179783FF05C087819085946090878783FC
:100DD00017968D919C91189793FF05C087819085F8
:100DE00084689087878317968D919C91189794FFBC
:100DF00005C08781908581609087878317968D9144
:100E00009C91189795FF05C0878190859064908785
:100E1000878317968D919C91189797FF05C08781BE
:100E2000908582609087878317968D919C91189703
:100E300096FF05C08781908590689087878311967B
:100E40008C911197818312968C91828308951396C9
:100E50002D913C911497C90184719C7084519C40E0
:100E600019F410924E012AC0C90184729C708452F8
:100E70009C4011F481E020C0C90184749C708454AA
:100E80009C4011F482E018C0C90184789C70845899
:100E90009C4011F483E010C0C90184709C7184509F
:100EA0009C4119F440934E0109C0C90184709C72A1
:100EB00084509C4219F485E080934E0120FF05C0C8
:100EC0008781908580619087878313968C91139793
:100ED00081FF05C087819085806490878783139602
:100EE0008C91139783FF05C08781908594609087CC
:100EF000878313968C91139784FF05C08781908513
:100F000081609087878313968C91139785FF05C026
:100F10008781908590649087878313968C9113972F
:100F200086FF05C0878190858260908787831396AE
:100F30008C91139787FF05C0878190859068908773
:100F4000878320914E01223009F44FC0233030F4C2
:100F5000222371F0213009F0F4C026C0243009F4B6
:100F60009AC0243008F460C0253009F0EAC0CAC035
:100F700013968C91139782FF05C0878190858468B2
:100F80009087878313968D919C91149793FF05C04A
:100F90008781908592609087878313968D919C912D
:100FA000149792FFD0C0C9C013968C91139782FFFB
:100FB00005C08781908590629087878313968D9175
:100FC0009C91149793FF05C08781908592609087CC
:100FD000878313968D919C91149792FFB4C087815B
:100FE0009085846890878783AEC013968C91139701
:100FF00082FF05C0878190859062908787831396D2
:101000008D919C91149793FF05C087819085926084
:101010009087878313968D919C91149792FF93C02C
:10102000878190859064DECF13968D919C91149763
:1010300092FF05C08781908590649087878313967F
:101040008D919C91149793FF05C08781908584684A
:101050009087878313968C91139782FF05C08781B1
:10106000908592629087878313968D919C911497B7
:1010700096FF05C08781908580629087878313964D
:101080008D919C91149795FF5CC0878190858860B5
:101090009087878356C013968D919C91149792FFE9
:1010A00005C08781908584689087878313968D918A
:1010B0009C91149793FF05C08781908592609087DB
:1010C000878313968C91139782FF05C08781908543
:1010D00090629087878313968D919C91149796FFC9
:1010E00005C08781908580629087878313968D9154
:1010F0009C91149797FF47C087819085886090875F
:10110000878341C013968D919C91149792FF05C0DF
:101110008781908590629087878313968D919C91AB
:10112000149793FF05C0878190859260908787838D
:1011300013968C91139782FF06C0878190859062E9
:1011400051CF243001F113968D919C91149794FF07
:1011500002C084E6848313968D919C91149795FF29
:1011600002C08CE9848313968D919C91149796FF0D
:1011700002C08CE9838313968D919C91149797FFFD
:1011800002C084E6838311968C9111978183129615
:101190008C918283089581E080936F010895EF928E
:1011A000FF920F931F93CF93DF93EC017B014130AC
:1011B0005105D9F489810A8187FD05C00E94D40EAA
:1011C000182F105E05C081950E94D40E10E2181BE6
:1011D00007FD04C0802F0E94D40E32C0802F81955D
:1011E0000E94D40E50E2581B45C08981EA814230EA
:1011F000510549F565E00E945812282F332727FD35
:1012000030958E2F65E00E945812992787FD9095A2
:101210002032310514F02FE130E08032910514F0D6
:101220008FE190E04FEF223E340714F421EE3FEFC0
:10123000EFEF823E9E0714F481EE9FEF122F105EB7
:10124000582F505E17C0992787FD909580589F4F63
:101250009595879595958795182F1F738E2F9927AC
:1012600087FD909580589F4F959587959595879583
:10127000582F5F732C81332727FD309520583F4F1F
:10128000E3E035952795EA95E1F72F718B81992752
:1012900087FD909580589F4F73E0959587957A9537
:1012A000E1F78F7190E063E0880F991F6A95E1F78D
:1012B000482F407C142BF7011083880F991F880F4B
:1012C000991F482F407C542B5183880F991F880FFA
:1012D000991F282B22838FEF8383888580958483B1
:1012E0008F8180958583DF91CF911F910F91FF9022
:1012F000EF9008952F923F924F925F926F927F925C
:101300008F929F92AF92BF92CF92DF92EF92FF9215
:101310000F931F93DF93CF93CDB7DEB76C970FB6C4
:10132000F894DEBF0FBECDBF87E088B983EC87B9E4
:1013300015B88FEF84B91BB88AB90E94990E4C0179
:101340000E94FF0E8B8F9C8F0E940E12898F9A8FA6
:101350008E01005F1F4F80E090E0B8010E94680599
:10136000C8018E010F5F1F4FB80140E050E00E949E
:10137000CF08EFE4F1E080E2DF011D928A95E9F702
:1013800080E091E0B801AF012BEC38E00E94850AC3
:10139000789400E010E0DD24CC24EE24FF2428EB38
:1013A000222E2BE0322E97E0A92EB12CAC0EBD1EC2
:1013B00080E1482E512C4C0E5D1E3E010894611CAC
:1013C000711C83B78E6083BF83B7816083BF8895AC
:1013D00083B78E7F83BF80916F018823E1F31092E2
:1013E0006F01C1010197F1F7DD2029F0B1E0DB16B3
:1013F00009F042C027C00E94FB108130910559F0CE
:10140000029791F4898D9A8D9C018901DD24D394F2
:10141000B2E0CB2E32C08B8D9C8D9C018901DD24E6
:10142000D394CC24C39429C0D4011296ED91FC919D
:1014300013970995D4011696ED91FC911797C50164
:1014400009951BC0D8011296ED91FC91139709954F
:10145000882341F00894E11CF11CBBE0EB16F10479
:101460005CF40BC0D8011696ED91FC911797C5015D
:101470000995EE24FF2401C0DD24C501B2010E94BC
:101480006805C201B3014C2D50E00E94CF08C30192
:101490000E947C0A96CF1092940210929302880FB9
:1014A0008093BA0085E48093BC00789408958823E3
:1014B00011F085EC01C085E88093BC000895282FC9
:1014C00030E070E088E090E0861B970BA90102C035
:1014D000440F551F8A95E2F7CA0102C0359527953A
:1014E0006A95E2F7822B0895863028F4E091710125
:1014F000F091720109950895A3E9B1E0FC0186E03D
:1015000001900D928150E1F708950F931F93182FCA
:10151000092F3093720120937101A3E9B1E0FB011F
:1015200086E001900D928150E1F710928302812FA5
:10153000902F9C01D9012AEF30E08D91F901ED56F1
:10154000FE4F80832F5F3F4F81E020303807A9F79F
:10155000DA0120E230E08D91F901ED56FE4F8083F3
:101560002F5F3F4F26323105B1F7459844981092CE
:1015700094021092930284EA8093BA0085E48093E7
:10158000BC0078941F910F9108952F923F924F9233
:101590005F926F927F928F929F92AF92BF92CF9203
:1015A000DF92EF92FF920F931F93DF93CF93CDB70C
:1015B000DEB768970FB6F894DEBF0FBECDBF48E622
:1015C000642E40E0742E882437E0232E312C2C0E1C
:1015D0003D1E28E0422E512CCBC084918D93319634
:1015E000A215B305D1F780E090E0FC01ED58FE4F65
:1015F000E081F0E0EE56FF4FE491ADE0B0E0AC0FDB
:10160000BD1FA80FB91FEC9301968A30910569F7A9
:10161000AA88CF8429812A2530E04C2D477050E0DC
:101620009E88B988C201841B950BB90102C0660F60
:10163000771F8A95E2F7CB0102C0359527954A9529
:10164000E2F7822B89198B258F83EE84DD842A8132
:101650002E2530E04D2D477050E0AC89C201841B2F
:10166000950BF90102C0EE0FFF1F8A95E2F7CF013B
:1016700002C0359527954A95E2F7822B8A198A2769
:101680008887EB892B812E2730E00D89077010E0C9
:10169000B201601B710BC901062E02C0880F991F91
:1016A0000A94E2F7002E02C0359527950A94E2F7D6
:1016B000822B8C198D2589872C812B2530E04A2F90
:1016C0004770842F90E0988F8F8BD888C2014F8904
:1016D000588D841B950BA90102C0440F551F8A9594
:1016E000E2F7CA010F8802C0359527950A94E2F700
:1016F000822B8D198C258A878D81E826FF24E7703F
:10170000F0E0C2018E1B9F0B970102C0220F331F16
:101710008A95E2F7C90102C0F594E794EA95E2F7E9
:101720008E298D198B258B878E81A827B0E0AD017E
:1017300002C0440F551F6A95E2F7BA0102C0B59581
:10174000A7950A95E2F76A2B6A1969256C87C1018A
:101750006DE771E046E050E00E947112009779F069
:10176000839466E070E0660E771E77E0871621F0BE
:10177000DE011196F30131CF109270013DC1282D89
:1017800030E02F5F3F4F522F442780918101FA01B3
:10179000E80FF11DEE56FF4F94912F5F3F4F322F10
:1017A000222780917601F901E80FF11DEE56FF4FD7
:1017B000E491E927E093830180917F01FA01E80F2A
:1017C000F11DEE56FF4F949180917801F901E80FD9
:1017D000F11DEE56FF4FE491E927E09384018091DB
:1017E0008201FA01E80FF11DEE56FF4F94918091AE
:1017F0007A01F901E80FF11DEE56FF4FE491E92758
:10180000E093850180917D01FA01E80FF11DEE560C
:10181000FF4F949180917501F901E80FF11DEE568B
:10182000FF4FE491E927E093860180917E01FA0160
:10183000E80FF11DEE56FF4F949180917701F90169
:10184000E80FF11DEE56FF4FE491E927E093870181
:1018500080918001FA01E80FF11DEE56FF4F94913F
:1018600080917C01F901E80FF11DEE56FF4FE491E4
:10187000E927E093880180917301FA01E80FF11DD7
:10188000EE56FF4F949180917901F901E80FF11D17
:10189000EE56FF4FE491E927E093890180917401AE
:1018A000FA01E80FF11DEE56FF4F949180917B01F4
:1018B000F901E80FF11DEE56FF4FE491E927E0939F
:1018C0008A0180917D01FA01E80FF11DEE56FF4F6C
:1018D000949180917401F901E80FF11DEE56FF4FCC
:1018E000E491E927E0938B0180918201FA01E80FEE
:1018F000F11DEE56FF4F949180917701F901E80FA9
:10190000F11DEE56FF4FE491E927E0938C018091A1
:101910008001FA01E80FF11DEE56FF4F949180917E
:101920007301F901E80FF11DEE56FF4FE491E9272D
:10193000E0938D0180917F01FA01E80FF11DEE56D1
:10194000FF4F949180917C01F901E80FF11DEE5653
:10195000FF4FE491E927E0938E0180918101FA0124
:10196000E80FF11DEE56FF4F949180917A01F90135
:10197000E80FF11DEE56FF4FE491E927E0938F0148
:1019800080917E01FA01E80FF11DEE56FF4F949110
:1019900080917B01F901E80FF11DEE56FF4FE491B4
:1019A000E927E093900180917601FA01E80FF11D9B
:1019B000EE56FF4F949180917801F901E80FF11DE7
:1019C000EE56FF4FE491E927E09391018091750174
:1019D000480F511D4E565F4FFA0194918091790145
:1019E000280F311D2E563F4FF9018491892780938E
:1019F000920181E08093700168960FB6F894DEBF83
:101A00000FBECDBFCF91DF911F910F91FF90EF904F
:101A1000DF90CF90BF90AF909F908F907F906F900E
:101A20005F904F903F902F900895982F805486306C
:101A3000A0F420E430E049E450E0FA01E21BF30BAB
:101A4000D901AD56BE4F8C91ED58FE4F80832F5F6C
:101A50003F4F2634310589F70895892F8654863003
:101A6000C8F48091D901809376018091DA01809346
:101A700075018091DB01809374018091DC0180937A
:101A800073018091DD01809382018091DE0180935A
:101A900081010895892F8C548430C8F48091DF012E
:101AA000809380018091E00180937F018091E1012A
:101AB00080937E018091E20180937D01892F90E0E7
:101AC000860F911D8035910511F40E94C50A089575
:101AD0001F920F920FB60F9211242F933F934F93A3
:101AE0005F936F937F938F939F93AF93BF93EF9386
:101AF000FF938091B90090E0887F907080399105C4
:101B0000E9F181399105D4F480379105A1F181374C
:101B1000910544F48036910571F18836910509F0FC
:101B2000B5C029C08038910549F18838910509F47C
:101B3000ADC08837910509F0A9C01DC0803B910553
:101B400009F463C0813B91054CF4803A910509F496
:101B500050C0883A910509F099C057C0803C910562
:101B600009F492C0883C910509F48EC0883B910528
:101B700009F08CC052C01092950286C080919502E7
:101B8000882351F12091BB00809170018823E1F0FE
:101B9000A0919302B0919402E0919302F09194028B
:101BA000E770F070E557FE4F8081E0919302F0916D
:101BB0009402E770F070ED57FE4F90818227890FF5
:101BC000AD56BE4F8C9352C0E0919302F0919402B7
:101BD000ED56FE4F20834AC08091BB0090E0909369
:101BE00094028093930281E0809395021092960272
:101BF0004BC0809193029091940220919602609143
:101C00009602821B0E94150D3FC080919302909115
:101C100094020E94740A10929602809170018823A7
:101C2000E1F0E0919302F0919402ED56FE4F808135
:101C3000E0919302F0919402E770F070ED57FE4F3F
:101C40002081E0919302F0919402E770F070E557E3
:101C5000FE4F9081821B892707C0E0919302F0918B
:101C60009402ED56FE4F80818093BB0080919302D9
:101C700090919402019690939402809393028091A4
:101C800096028F5F8093960285EC01C085E8809371
:101C9000BC00FF91EF91BF91AF919F918F917F9188
:101CA0006F915F914F913F912F910F900FBE0F90C9
:101CB0001F901895419A80E38A95F1F7419880E04A
:101CC00090E030E048E1242F2A95F1F740983695CE
:101CD000329B3068242F2A95F1F7409A019688307C
:101CE000910589F73093980280E090E048E1242F35
:101CF0002A95F1F740983695329B3068242F2A9523
:101D0000F1F7409A01968830910589F7309399024E
:101D100080E008951F931FB7F894399A389A3A983B
:101D2000429A409A41980E945A0E1FBF80E01F912C
:101D3000089586E091E00895FC01009719F1209143
:101D4000980280919902482F50E0CA01807F9070DC
:101D5000803F910521F481E08093970202C01092A8
:101D6000970280919702882321F083E0808321836A
:101D700009C082E08083942F882730E0822B932B48
:101D800092838183809198029091990290939B0213
:101D900080939A02089588E992E06AE972E042E04D
:101DA00050E00E94711208958823A1F0E3E1F1E070
:101DB00021E0482F552747FD5095808190E0481736
:101DC00059071CF4822F815008952F5F31962032DD
:101DD000A1F78FE1089520913E01253079F022236B
:101DE00069F0892B31F0233049F082E080933E0185
:101DF0000895213019F084E080933E01089582E334
:101E000091E00895CF92DF92EF92FF921F93DF93BC
:101E1000CF930F92CDB7DEB785E080933E0110E0FF
:101E20008CE2C82E81E0D82E7E010894E11CF11CC2
:101E300012C0F6013197F1F70197D9F71982C7015E
:101E400061E070E00E944810489741F01F5F1F302A
:101E500011F480E004C08CE291E0EBCF81E00F90C0
:101E6000CF91DF911F91FF90EF90DF90CF90089579
:101E7000009741F0DC01ECE9F2E089E001900D927D
:101E80008150E1F7A5EAB2E0ECE9F2E089E00190E7
:101E90000D928150E1F708958CE992E065EA72E0D5
:101EA00049E050E00E94711208951F93DF93CF9391
:101EB000CDB7DEB7A6970FB6F894DEBF0FBECDBF85
:101EC0001982CE01019661E070E00E9448108831CD
:101ED00019F010923E016DC08091DA02882331F032
:101EE00080913E01853011F410923E018091DA021A
:101EF000882319F485E080933E0180913E01823071
:101F0000E9F08430A1F1882309F049C083E0898396
:101F100080E88A8381E08B83CE01049660E870E0DC
:101F200042E250E00E947E12CE01019663E270E030
:101F30000E944810882399F184E02FC013E0198390
:101F400080EC8A838BE18B83CE01049661E070E0A4
:101F500040E250E00E947E12CE01019663E270E002
:101F60000E9448108823D9F010933E0118C083E0E6
:101F7000898380EC8A838BE18B8380E2FE01349637
:101F8000DF011D928A95E9F7CE01019663E270E0C8
:101F90000E944810882319F081E080933E0181E07F
:101FA0008983CE01019661E070E00E944810803282
:101FB00011F08FEF5AC084E080939C0220E030E063
:101FC00040E050E061E070E0F901ED53FD4F8081A9
:101FD000882349F0CB01022E02C0880F991F0A9472
:101FE000E2F7482B592B2F5F3F4F2031310561F726
:101FF0005093A00240939F0219821A8240E020E091
:1020000030E060E870E0F901ED52FD4F80818823F7
:1020100039F0CB01022E02C0959587950A94E2F71C
:10202000482B2F5F3F4F2830310569F749834A819C
:1020300020E030E060E870E0F901E552FD4F80817A
:10204000882339F0CB01022E02C0959587950A941A
:10205000E2F7482B2F5F3F4F2830310569F7898120
:1020600080939D0240939E0280E0A6960FB6F8945E
:10207000DEBF0FBECDBFCF91DF911F9108950E94AB
:10208000550F80E008953B984398249A2C98089522
:10209000EF92FF920F931F93CF93DF937C01662300
:1020A00009F456C070E020E030E0E0E0F0E011C05C
:1020B00088818423FD01ED53FD4F80831196469561
:1020C000A017B107A9F72F5F3F4F2617370754F422
:1020D000FD01DF0140E8E701C20FD31F8F01085F58
:1020E0001F4FE6CFE3ECF2E0CF93DF93EF93FF9344
:1020F0000191002311F069F41BC000003B9A1DE020
:1021000014D03B980000000000000000119781F7F8
:102110000FC03B9A12E0000008D03B9819E005D0B0
:1021200000000000119721F703C01A95F1F70895F8
:1021300000000000FF91EF91DF91CF913B9A12E0F8
:102140000000F3DF3B980FEF0A9511F0339BFCCFB3
:10215000E3ECF2E0EF93FF93112700270395A1F042
:102160003399FCCF08C00BE4039572F03399FCCF90
:10217000139551F001930BE4039532F0339BFCCFA0
:10218000139511F00193EFCFFF91EF91612F70E064
:102190006115710531F110FF24C040E050E020E0EE
:1021A00030E00CC08081F901EE53FD4F9081E0E0FA
:1021B000891708F4E1E0EC934F5F5F4FDA01AD530C
:1021C000BD4FF901ED53FD4F2E5F3F4F411750F3C7
:1021D00084E18A95F1F79B01215030403595279590
:1021E00002C020E030E0C901DF91CF911F910F9133
:1021F000FF90EF900895DF93CF930F92CDB7DEB7A6
:102200001982CE01019661E070E00E9448100097AB
:1022100019F420E030E026C0489711F58091C702FC
:10222000882311F098E001C090E08091C8028111EC
:1022300094608091C902811192608091CA028111DB
:1022400091609A3028F4983028F4953049F405C00C
:102250009B3031F422E030E005C021E030E002C0E4
:1022600023E030E0C9010F90CF91DF91089585E020
:102270008093AF0220E030E040E050E061E070E0A9
:10228000F901ED53FD4F8081882349F0CB01022EE7
:1022900002C0880F991F0A94E2F7482B592B2F5F31
:1022A0003F4F2031310561F75093B7024093B6029A
:1022B00020E030E050E060E870E0F901ED52FD4FC1
:1022C0008081882339F0CB01022E02C09595879535
:1022D0000A94E2F7582B2F5F3F4F2830310569F7FA
:1022E00020E030E040E060E870E0F901E552FD4FA9
:1022F0008081882339F0CB01022E02C09595879505
:102300000A94E2F7482B2F5F3F4F2830310569F7D9
:102310008091AE02882381F08091C102581B5093B6
:10232000B0028091C202481B4093B10240E020E01D
:1023300030E060E870E00CC05093C1024093C202EC
:102340001092B0021092B10281E08093AE02EECF03
:10235000F901ED51FD4F8081882339F0CB01022E28
:1023600002C0959587950A94E2F7482B2F5F3F4F5F
:102370002830310569F74093B20240E020E030E0B8
:1023800060E870E0F901E551FD4F8081882311F08C
:1023900080E007C0CB01022E02C0959587950A9474
:1023A000E2F7482B2F5F3F4F2830310559F7409314
:1023B000B30240E020E030E060E870E0F901ED5069
:1023C000FD4F8081882339F0CB01022E02C0959504
:1023D00087950A94E2F7482B2F5F3F4F283031054D
:1023E00069F74093B40240E020E030E060E870E03C
:1023F000F901E550FD4F8081882339F0CB01022E91
:1024000002C0959587950A94E2F7482B2F5F3F4FBE
:102410002830310569F74093B50208958FE391E0C4
:102420000895009741F0DC01EFEAF2E089E00190C5
:102430000D928150E1F708958FEA92E068EB72E027
:1024400049E050E00E9471120895DF93CF93CDB719
:10245000DEB728970FB6F894DEBF0FBECDBF80E47D
:10246000898383E08A831B82CE01019663E070E05A
:102470000E944810803411F081E003C00E9437119F
:1024800080E028960FB6F894DEBF0FBECDBFCF9187
:10249000DF9108951092AE020E94251290E08823E9
:1024A00009F491E0892F08950E94251280E0089593
:1024B00087FB082E062687FD819567FD619505D06F
:1024C0000EF4919507FC81950895991B79E004C05D
:1024D000991F961708F0961B881F7A95C9F7809563
:1024E0000895FB01DC0104C08D910190801921F455
:1024F00041505040C8F7881B990B0895DC0101C07A
:0E2500006D9341505040E0F70895F894FFCFDE
:10250E000000A42001018A0E5A0ECB0E9C0E000074
:10251E00000000010203060C1217222F3C43474B0A
:10252E004E51535400000000000000000000000057
:10253E0000003F10550F4C0F380FEB0E020F0554D5
:0C254E001225121C12111200004A12008B
:00000001FF
